:020000040000FA
:1000000083016B2800000000F200030E8301F3005F
:100010000B1183120313AA0F0E28AB0AB10F11287C
:10002000B20AB60F1428B70AB80F1728B90ABA0FC0
:100030001A28BB0ABC0F1D28BD0ABE0F2028BF0A04
:10004000C00F2328C10AC20F2628C30AC40F2928BB
:10005000C50A730E8300F20E720E09008B138B1B00
:100060002E2871088A007008820000088316031386
:100070009A001C158B138B1B3A2855309D00AA3013
:100080009D009C148B179C1843281C119B0A840A02
:10009000F00B35280800831603131C141A0880007F
:1000A0009B0A840AF00B4B280800003083160313C8
:1000B0009B0083130230F0002030840035200800BC
:1000C0000030831603139B0083130230F0002030AE
:1000D00084004B20080020308B00831203138030F3
:1000E0008500003086008F30831681003F30850008
:1000F00000308600831207309F0083132030840075
:100100008001840A841F802884168001840AF030CC
:100110000402031D85288317203084008001840A8F
:1001200050300402031D8E286020831203138101C6
:100130000B118B1783120313A71CA028A301AE2851
:1001400083120313281CAE282418AE282414271861
:10015000AB28A30AAE2883120313A303831203134D
:100160002818B32824109B30F0000230F1008312CD
:1001700003130310230DF0070318F10A2E20831236
:100180000313A500F00A0319F10A2E2083120313AA
:10019000A6008B172518CE282711CF282715A518BC
:1001A000D328A813D428A8172519D8282910D92866
:1001B0002914A519DD28A910DE28A914251AE2287A
:1001C0002911E3282915A51AE728A911E828A91556
:1001D000251BEC282912ED282916A51BF128A711AB
:1001E000F228A7152719F828A71DFB282714FB2894
:1001F0008312031327100030831203132B02031DF5
:10020000032914302A02031C10290030AB021430D9
:10021000AA02031CAB03271A0F292716102927123D
:1002200083120313A81C1729AC01AD012A298312DC
:100230000313271E2A292E182A292E14A71A242927
:10024000AC0F2A29AD0A2A2983120313AC032C0F01
:100250002A29AD0383120313271A2F292E10831284
:100260000313A712051C39292F1839292F14271712
:100270003F2983120313271305183F292F108312D8
:100280000313A81D4629A001A101592983120313B4
:10029000271F5929301859293014A71B5329A00F9B
:1002A0005929A10A592983120313A003200F5929A0
:1002B000A10383120313271B5E293010831203133B
:1002C000A7132008F0002108F100A81C6D290030B8
:1002D000F1020030F002031CF103710883120313D2
:1002E0002D02031D752970082C0283120313031CB1
:1002F0007B29A8147C29A810B318862933189229C1
:10030000281D9229B101B201B314281400308312C0
:1003100003133202031D8E2904303102031C92297B
:10032000B310281083120313281D982933149B2916
:10033000831203133310A8189F292811A2298312AE
:1003400003132815271BA829221CA8292210552091
:1003500083120313271FAD292214073020028312B2
:100360000313031DB529A815B629A811281EBA29FB
:100370000517BD29831203130513281AC1298517F0
:10038000C429831203138513281FC829B401D62951
:1003900083120313271CD6293518D6293514A81A19
:1003A000D329B40AD62983120313B4038312031387
:1003B0002718DB29351083120313A812281BE22902
:1003C0000230E32902303402031CE8292817E92906
:1003D00028133408013C83120313031CF329031967
:1003E000F3292816F4292812271DFA29B601B70186
:1003F0000616072A83120313061E072A0030370247
:10040000031C072AC3303602031C072A0612831274
:100410000313A81F0F2AB801B90186161C2A8312DC
:100420000313861E1C2A00303902031C1C2AC33009
:100430003802031C1C2A861283120313291C242A47
:10044000BA01BB010617312A83120313061F312A92
:1004500000303B02031C312AC3303A02031C312A0C
:10046000061383120313A91C392ABC01BD01861788
:10047000462A83120313861F462A00303D02031CBE
:10048000462AC3303C02031C462A861383120313F8
:10049000291D4E2ABE01BF0186155B2A8312031354
:1004A000861D5B2A00303F02031C5B2AC3303E02DC
:1004B000031C5B2A861183120313A91D632AC00142
:1004C000C1010615702A83120313061D702A00301D
:1004D0004102031C702AC3304002031C702A06111B
:1004E00083120313291E782AC201C3018614852AA8
:1004F00083120313861C852A00304302031C852ABD
:10050000C3304202031C852A861083120313A71DE1
:100510008D2AC401C50106149A2A83120313061CEE
:100520009A2A00304502031C9A2AC3304402031C55
:100530009A2A06109A280134003402340034043414
:100540000034083400341034003420340034403493
:100550000034803400340034013400340234003478
:06056000043400340834ED
:084000000000010000000000B7
:02400E00183F59
:1042000000000000000000000000000000000000AE
:10421000000000000000000000000000000000009E
:10422000000000000000000000000000000000008E
:10423000000000000000000000000000000000007E
:10424000000000000000000000000000000000006E
:10425000000000000000000000000000000000005E
:10426000000000000000000000000000000000004E
:10427000000000000000000000000000000000003E
:10428000000000000000000000000000000000002E
:10429000000000000000000000000000000000001E
:1042A000000000000000000000000000000000000E
:1042B00000000000000000000000000000000000FE
:1042C00000000000000000000000000000000000EE
:1042D00000000000000000000000000000000000DE
:1042E00000000000000000000000000000000000CE
:1042F00000000000000000000000000000000000BE
:00000001FF
